:020000040000FA
:060000000219FD020310CD
:03001300020501E2
:03001B0002008D53
:03002B000202D5F9
:03005B000205108B
:030073000202FD89
:100080000406080C10182030406080A0C0C2AFC227
:10009000A853E6EFC28E856B8BC0D0D2D3C0E0C030
:1000A000F0C2CAA8CCA9CDD2CAD2AF758A00C3E823
:1000B000956CF8E9956DF9C3E913F9E813F8E5666D
:1000C0006007C3E913F9E813F8E97025E8956E4075
:1000D00020956E501CE582B410177C007B007A00DE
:1000E0007908900000A86AE5667004C3E813F80177
:1000F000FA900000D2A8D2AA61BAE0FDC39CC398CE
:1001000040EF98EB33FB0582E0FCC39DC39840E1D0
:1001100098EB33FB0582E0FDC39CC39840D398EB7A
:1001200033FB0582E0FCC39DC39840C598EB33FBCD
:100130000582E0FDC39CC39840B798EB33FB058272
:10014000E0FCC39DC39840A998EB33FB0582E0FD1A
:10015000C39CC398409B98EB33FB0582E0FCC39D96
:10016000C398408D98EB33FB05822175900000D237
:10017000A8D2AA61BAE0FDC39CC39840EF98EA33C5
:10018000FA0582E0FCC39DC39840E198EA33FA0582
:1001900082E0FDC39CC39840D398EA33FA0582E01D
:1001A000FCC39DC39840C598EA33FA0582E0FDC3BD
:1001B0009CC39840B798EA33FA0582E0FCC39DC31C
:1001C0009840A998EA33FA0582E0FDC39CC39840A1
:1001D0009B98EA33FA0582E0FCC39DC398408D9852
:1001E000EA33FA0582EBC46B6A54F0F9EAC454F0BE
:1001F000C3996009900000D2A8D2AA61BAEBF4C4F6
:1002000054F0F9EAF4C4540F49FAEBF4C4540FFB68
:10021000C3EAF99460FAEB9400FB5020C3E97B0039
:100220007A0079006016C3135006F9C39552600A2C
:10023000E9F552755300790080020553303A27C31F
:10024000EA94D0F8EB9407F9400BE8FAE9FB203583
:1002500009D235415A303502C235203902B235C390
:10026000EA33FAEB33FBEB2B3B3BF9C3EB13FBEA33
:1002700013FAEA29FAEB3400FB30E3047AFF7BFF40
:10028000E5255403601B202A18E55D33F9EB700760
:10029000C3E99A4002E9FAE53CC4332AFAEB340098
:1002A000FBC3EA33C4540FF8EB33C454F048F8707E
:1002B00005EA60027801C3EB13FBEA13FA90000031
:1002C000D2A8D2AAE52260021522819E900000D217
:1002D000A8D2AA61BAC0D0C0E0C2CF0541E5236070
:1002E000021523C3E554600575550041F8E5552412
:1002F00001F55550037555FFD0E0D0D032C2AF5351
:10030000E67F7592FA7593FFC22053917FD2AF3288
:10031000C0E0E58A303408856B8BF0A3D0E032D0A2
:10032000E0C2AF53E6EFC0D0C0E0C0F0D2D3D2AF4E
:100330005388EFA88AA98C758A00758C00438810B1
:1003400030331FE8C4540FFAE9C454F04AFAC31317
:100350002AFAC3E833F8E933F9E82AFAE93403FB67
:1003600061AB30320FC3E833E933FAE82AFAE934F3
:1003700000FB61AB303115E875F056A4AAF0E975C1
:10038000F056A42AFAC5F03400FB61ABE875F02BF7
:10039000A4AAF0E975F02BA42AFAC5F03400C3131F
:1003A000FBEA13FAC3EB13FBEA13FAC3EB9409500D
:1003B00009C3EA949AEB940350160522E5227002D1
:1003C0001522C3E5229432500281F475540081F75E
:1003D000E522600215223036067C007D0461EAAC1D
:1003E00031AD32303A04AC33AD34C3EA9CFAEB9D04
:1003F000FB9208AE60AF61303A425007203509D217
:10040000358108303502C235303504AE62AF632025
:100410003902B235C3EA33FAEB33FBA208500AEAD9
:10042000F42401FAEBF43400FBC3EA9428FAEB94C9
:1004300000FB501478007A007B008148A208500825
:1004400078007A007B00819EE52554036019202AFC
:1004500016E55DF9EB7007C3E99A4002E9FAE53C5D
:10046000C42AFAEB3400FBEA8EF0A4F9AAF0EB8E72
:10047000F0A42AFAC5F03400FBC3EB13FDEA13F82D
:100480000FEF146004C3E833F8C3E933EA33FAEB3F
:1004900033FBDFEDEB30E20678FF7AFF7B03885415
:1004A000D230E86003755500C3E55BFC955C400203
:1004B000AC5CC3EC95545008EC75F004A4FAABF0B6
:1004C000EAF4F8EBF45403F98856895775230AE5E2
:1004D0005A30E110D0F0D0E0D0D053F7DF43F740EE
:1004E00043E61032D0F0D0E0D0D053D8FE43DA014A
:1004F00043E6103275230AD0F0D0E0D0D043E610A6
:1005000032C2AAD28EC2CA85CC6C85CD6DD2CA3217
:10051000C2AFC0D0C0E0D2D38556FB8557FC85570B
:100520005A53F7BF53DAFED2A8303402D2AA53E6A8
:10053000EF53F7DF53D8FED0E0D0D0D2AF327901FD
:10054000801479038010790A800C791E8008796400
:10055000800479C880007817E4D5E0FDD8FAD9F690
:100560002278FF20282879A1E76023E548601F74DE
:10057000FF8548F084853FF030290375F005A4F825
:10058000C5F0600278FFC3E8955D5002A85D885C05
:1005900022C3E54794E4E5489400E55C500314A1C8
:1005A000A2046002F55C2275E89022055EC3E55E58
:1005B0009408405330EDF4A8BDA9BE755E00E9FA79
:1005C00079A0E76041EA7006E55F6018800CC3E837
:1005D000955F600EE55F5005600A1480070460FABD
:1005E0008002E55FF55FC39569401B755BC0C394EE
:1005F000044013755B80C39404400B755B40C39447
:10060000044003755B0022E55B2410500274FFF583
:100610005B22743279A687F0A4C5F0A2F733F55DAA
:10062000227547007548F022C2AFC2CAA8CCA9CD36
:10063000AA4130CF010AD2CAD2AFAB42AC43884202
:100640008943C3E89BF8E99C202808F9302C02E193
:1006500038C191AD448A44F9EA9DFA600678FF7981
:10066000FFC176AE45AF468B458C46A842A943C331
:10067000E89EF8E99FF9C3E54813FBE54713FAE85C
:100680002AF547E93BF54850067547FF7548FFC115
:10069000DEAA47AB48AC47AD487E047F02C3EB946B
:1006A00004400D1E1FC3EB940840052029021E1FA5
:1006B000C3ED13FDEC13FCDEF7C3EA9CFAEB9DFBE4
:1006C000EF6009C3E913F9E813F8DFF7EA28FAEB5A
:1006D00039FB8A478B4850067BFF8B478B48C3EB1F
:1006E00094025002D22C3028047F03E1097892E66C
:1006F000FFC3E53D948240110FC3E53D94A0400146
:100700000FC3EF940640027F057E02E548C4540FF4
:10071000F9E548C454F0F8E547C4540F28F8C3E895
:100720009EFAE99400FB4009C3EA9401EB9400505F
:10073000047A01E4FB020784AA47AB48EBC4FEEA53
:10074000C4540F4EFCC3EA9CFAEB9400FBC3E813BD
:10075000C313F8EA28FAEB3400FB8A478B48C3EB53
:1007600094024002C22C7802EBC4FE7B00EAC4541F
:100770000F4EFAC3EA98FA4005C3940150027A0179
:100780007892E6FF302002E184854E92854F93D225
:100790002043E680C3E49AF8E49BF9302C03020876
:1007A00012E8FAE9FBD3E913FDE813FC884E894F00
:1007B000C3EF94036038EF20E00CE82CF8E93DF932
:1007C000ECFAEDFB8013E828F8E939F9C3E82401D5
:1007D000F8E93400F97AFF7BFFC3EF9403400F8AF6
:1007E000508B51884A894B8C4C8D4D02084788505C
:1007F00089518A4A8B4B8C4C8D4D3028127550F0A4
:100800007551FF754CF0754DFF754EF0754FFF0239
:100810000847E8FAD3E813FC884EC3EF940360213D
:10082000EF20E007E82CF8ECFA0132E8282401F880
:100830007AFFC3EF940340098A50884A8C4C02081F
:100840004788508A4A8C4C3020020147753A02D2C0
:100850002043E680E52554036034A847A948C3E94E
:1008600013F9E813F8C3E913F9E813F8302804E999
:100870002440F9C2AF53E67F759100C3E498F59424
:10088000E499F595759104D22043E680D2AF22D247
:1008900021754900752000302B0375204001ADD231
:1008A00021754900752040302B03752000780179AF
:1008B00001202C20E52554036002C2217914E5486B
:1008C000C313700104F8C394144002781430280450
:1008D000781B791B202010E549600C302803D53A9D
:1008E00004D2222154114F0549E59B5440B5200202
:1008F000213E30280908C3E89940011801D420217D
:100900000A08C3E899400201AD01D4C22153E67F31
:10091000759100302C117594007595F8759104D27D
:100920002043E6800208ADE5487EFFC3334005C39F
:10093000334001FEC3E49E759400F595211CC3E588
:10094000399401500201AD30210201ADD80221528B
:1009500001D4C222C2AF53E67F75910085509485C1
:100960005195759104854A92854B93D22043E68038
:10097000D2AFE525540360072029020539801030E5
:10098000220D202B0A2021071581158102137522C3
:1009900078003021027801E53D75F007A4F9E5F013
:1009A00028F5F0E9A2F013A2F113A2F213F53DC36A
:1009B00094785003753D78C3E53D953E4009C29358
:1009C000C294C29575D57F30200221C7854C92858F
:1009D0004D93D22043E68022203814C2AFC294C285
:1009E00090D293D29575D53BD2AF759F2341D8C293
:1009F000AFC294C292D295D29375D53ED2AF759FB5
:100A00002341D8203814C2AFC295D29475D53DC2C7
:100A100090D293D2AF759F1341D8C2AFC293D294F4
:100A200075D53DC292D295D2AF759F0341D820387B
:100A300014C2AFC293C292D295D29475D53DD2AFB3
:100A4000759F0341D8C2AFC295C290D293D294751C
:100A5000D53DD2AF759F1341D8203814C2AFC29490
:100A6000D29375D53EC292D295D2AF759F2380683E
:100A7000C2AFC294D29575D53BC290D293D2AF7516
:100A80009F238054203814C2AFC295C291D294D211
:100A90009375D53ED2AF759F13803DC2AFC293C24E
:100AA00091D294D29575D53BD2AF759F0380292002
:100AB0003814C2AFC293D29575D53BC291D294D2AD
:100AC000AF759F038012C2AFC295D29375D53EC257
:100AD00091D294D2AF759F13227A147B7880127AC8
:100AE000107B8C800C7A0D7BB480067A0B7BC880DF
:100AF00000E564D5E001227902E4C294D5E0FDD29C
:100B000091D294D5E0FDC294D5E0FDC291D294D5A6
:100B1000E0FDE920E004D290D29330E004D292D2FA
:100B200095E564D5E0FDE920E002C29330E002C221
:100B3000957496D5E0FDD9C1EAF8D5E0FDD8FBDB88
:100B4000B0C29422C293C294C295C293C294C29579
:100B500075D57F22788076FF0876FF0876FF0876C5
:100B6000FF0876FF0876FF0876090876FF08760109
:100B7000788C76010876FF0876FF0876FF0876FF06
:100B80000876FF0876030876FF0876FF0876FF08E8
:100B900076250876D00876280876500876040876F8
:100BA000FF0876020876FF08767A0876FF0876074F
:100BB0000876010876FF0876FF087600087600229E
:100BC000FA75F00CA4ABF0EAC333F8740133F9E81A
:100BD000C333F8E933F9E8C32BF8E93400F9227894
:100BE00088E6C39403D23A5002C23AC238E630E1F2
:100BF00002D238A23892397886E614900080937831
:100C0000A6F67886E6F53FC394025003753F027856
:100C10009CE6753EFFB40203753EA0B40303753E27
:100C20008278A0E6F8600674282409D8FCF5697873
:100C300096E671C088318932789EE671C088338922
:100C4000347897E671C08835893671442230361180
:100C50007A007B007CFF7D007E0091B38B618A600F
:100C600022303A227896E6FA7B00789EE6FC7D00F8
:100C7000C3EA33FAEB33FBC3EC33FCED33FD7E0AFE
:100C800091B38B638A627896303A02789EE6FA7B5B
:100C9000007897E6FC7D007E00303A10C3EA33FA14
:100CA000EB33FBC3EC33FCED33FD7E0A91B38B6178
:100CB0008A6022C3EC9EFCED9400FDC3EC9AFCED2F
:100CC0009BFDC3EC9423ED940050047C237D00C372
:100CD000EC94FFED940140047CFF7D017BFF0B7AD7
:100CE000000AEA7009C3EC33FCED33FD81DEEC8AC7
:100CF000F0A4AEF0ED8AF0A42E947C40E4EAF46017
:100D0000DD22D236914D12054A12054A7A007B0047
:100D10007C10120542E5542AFA74003BFBDCF37C9C
:100D200004C3EB13FBEA13FADCF7FFEB60027FFF6F
:100D3000C236914D2278A5E6F95403C2857002D2DD
:100D400085E9540CC2867002D286E95430C287709D
:100D500002D287E954C0700022756700756800757B
:100D600097DE7597AD7581C043FF8075EF0675A955
:100D70000071447580FF75F1F075A4E07580FF7512
:100D8000D4FF75900075F23F75A53F75900075D53D
:100D90003F75A60175E34075E2027144E4F8F6D8A8
:100DA000FD71541213B178988664753001C2AF1288
:100DB000055251D912054A51DF12054A51E5120573
:100DC0004AB135C2AF75670075680078FA79FA30B4
:100DD0008407D9FBD8F7021C0071DF914D78988603
:100DE00064714475E404758811758E0475890975FC
:100DF000C80475910475D84075D90875F782759E39
:100E00000075960275DA4A75DB0075A82175E690C3
:100E100075B801759B80759D0075D10C75BC5975B1
:100E2000BB1075E88075B20112053ED2AF753C006B
:100E3000C230120552C231C232C233C234755200BE
:100E400075530075220012054EC3E522940A500224
:100E5000E11AD23175220012054EC3E522940A50E0
:100E600002E11AC231D23275220012054EC3E522C8
:100E7000940A5002E11A75E4C4758851758E0175A3
:100E800089AA758C00758D00C2A9D2ABD2AA756BE8
:100E9000C0756A14756E50C232D23475220A1205BA
:100EA0004E756A10C3E522940A75520075530040CE
:100EB00069758E0C756B80756A28756E2875220AA7
:100EC00012054E756A20C3E522940A7552007553C7
:100ED000004047758E0C756BC0756A14756E14757D
:100EE000220A12054E756A10C3E522940A75520053
:100EF000755300402575E404758811758E04758955
:100F000009D2A9C2ABC2AAC234D2337522001205DB
:100F10004EC3E522940A4002A1C3120542203003C9
:100F2000020DC3C2AF51D951D951D9D2AF12055216
:100F3000203403303A03020FD8120542788CE6C3FE
:100F400094015002E1D8E530C394015002E1D87514
:100F500067A57568F17F02D236914D12054EC2AF7A
:100F6000C236914DC3E554947FD2AF406B12053E1B
:100F7000C2AF51EBD2AFDFDFB102C3EF7897F61209
:100F8000055212149E7F0AD236914D12054EC2AF01
:100F9000C236914DC3E554947FD2AF50E812053E5E
:100FA000C2AF51D912054651D9D2AFDFDAB102EF43
:100FB00024037896F6F87997E7C394234003985072
:100FC00006E824237897F61205521213F81214CD6E
:100FD00012054E914D020DC375670075680012052C
:100FE0004EC3E55494014002E130C2AF51EB51EBE6
:100FF00051EBD2AF120552753000E4F537F53805E4
:1010000037E537F4703F0538789AE678191460129E
:10101000783214600D787D14600878FA14600375D6
:101020003800C3E53898401D120B4412053E1538B0
:1010300075370078998664C2AF120AEBD2AF789800
:10104000866412054E120546E5237003020DC3C3E4
:10105000E5549401500AC3E55294015016020FFF63
:1010600012054EE5237003020DC37552007553003F
:10107000021215C3E55294017017C2AF120B4478E7
:10108000998664120AD978988664D2AF12054E41C7
:1010900007C3E55294027017C2AF120B44789986C9
:1010A00064120ADF78988664D2AF12054E4107C3F6
:1010B000E55294037017C2AF120B447899866412FC
:1010C0000AE578988664D2AF12054E4107C3E5520F
:1010D00094047017C2AF120B4478998664120AEB1D
:1010E00078988664D2AF12054E4107C3E552940545
:1010F0007017C2AF120B4478998664120AEB789885
:101100008664D2AF12054E4107C3E55294077019A9
:10111000C3E55394065002014F7401303A02740340
:101120007888F6C238C2394107C3E552940870196D
:10113000C3E55394065002014F7402303A0274041E
:101140007888F6D238D2394107C3E552940970172E
:10115000C3E55394065002014F303A0BC37888E63A
:101160009402F6C23A4107C3E552940A7016C3E5E9
:101170005394065002014F203A0A7888E62402F67A
:10118000D23A4107C3E55294147025C3E55394063F
:101190005002014FC2AF901A0B740093D2AF7888FF
:1011A000F613C238C2394002D2384002D2398057D1
:1011B000C3E55294157038C3E5539406404FC2AF4F
:1011C000901A0B740093D2AFF8B801027402B802FF
:1011D000027401B803027404B8040274037888F638
:1011E00013C238C2394002D2384002D2398018C303
:1011F000E552940C70117567A57568F1C3E55394B9
:1012000006400A71F8D2AF75520075530075670039
:10121000756800014FC2AF120B44E4D2AFE4F55E33
:10122000F524F525F53D755E0812053E1205A7303B
:10123000EDFDA8BDA9BEE97001F8885F1205AB7588
:101240005E08C2AF120612855D5B855D5CD2AF3071
:101250003A07C238303502D238D228753900120A1E
:1012600084120AAF1206211206281206211206283D
:1012700012062112089F1209901209D8120628128C
:10128000088F202C03120561302C031205911209DE
:1012900090120A0312062812089F120990120A2EB1
:1012A00012062812088F120990120A5912062812E3
:1012B000089F120990120A841206281205A7120824
:1012C0008F120990120AAF1205AB12062830282798
:1012D000855D5B79187A0CC3E53999400EC228D236
:1012E000298A3B855D5B855D5C800CC3E554940178
:1012F0004003021273617D30291F202B1CE53B1433
:101300007006C229D22A4173F53B203A07C3E5543F
:10131000940140030212738064753C00203A0F78F8
:10132000FA79A4E760027803C3E55598504FE523A6
:10133000604B303A17203805203507800F303502D2
:10134000800A202B07D22B855D5B41A378F0302BE0
:1013500005855D5B7820C3E5489850030212733021
:101360002B1BC22BC238303502D238D229753B1222
:10137000855D5B4173053CE55460026180753C000E
:10138000C2AF120B44752400752500D2AF12054E72
:10139000120B4478A4E6600CC290D293C291D2940E
:1013A000C292D295C3E53C94044003020DC3020FE0
:1013B000FA901A0D78209131E520B4550AA39131A5
:1013C000E520B4AA0280137567A57568F1120B5465
:1013D00071F8756700756800801D901A0378807B2E
:1013E0000A9131A308DBFA901A0F788C7B1A91319D
:1013F000A308DBFA901A2922C2AF91749151901A76
:101400000074109136A374079136A374219136901D
:101410001A0378807B0A9135A308DBFA901A0F78BB
:101420008C7B1A9135A308DBFA91879165901A2974
:1014300022E493F622E6438F01538FFDFFC3E58339
:10144000941C400122EF8567B78568B7F0538FFE83
:1014500022438F02438F018567B78568B7901A0DC5
:10146000F0538FFC22901A0D74559136901A0E7419
:10147000AA9136227A3079D07820901A409131E5BD
:1014800020F709A3DAF7227A3079D0901A40E79151
:101490003609A3DAF9227C05120552DCFB22C2AF21
:1014A000120AD9120ADF120AE5120AEB12054612D5
:1014B0000AD9120ADF120AE5120AEB120546120ACD
:1014C000D9120ADF120AE5120AEBD2AF22C2AF121A
:1014D0000AEB120AE5120ADF120AD9120546120AAD
:1014E000EB120AE5120ADF120AD9120546120AEBBC
:0C14F000120AE5120ADF120AD9D2AF225C
:1019FD00020D59100721FFFFFFFFFFFF09FF01FF38
:101A0D0055AA01FFFFFFFFFF03FFFFFF25D0285061
:0D1A1D0004FF02FF7AFF0701FFFF0000FF3A
:101A4000234A5F4C5F30302320202020202020209C
:101A500023424C48454C492445464D3842313023B9
:101A60002020202020202020202020202020202076
:101C0000C2AFC2D37597DE7597AD7581C075A90057
:101C100043FF80752438752503B1DB7529A5752A26
:101C2000F143F11053A4EFD28475D4FF75E3407DE6
:101C3000FA780379E67C10752200752300901DE880
:101C40007B0675249875250130840281482084081C
:101C5000D8FBD9F9DCF781BA308408D8FBD9F9DC94
:101C6000F781BAB19BE493A3C39A6004DDC381BA40
:101C7000DBDBB18D600281317B08E493FAA3B16EA6
:101C8000DBF87A30B16E752200752300B18DEAFC65
:101C9000EBFDC3ED94FE400EB18D8A278B28ED300D
:101CA000E0048A828B83B18D7AC270D8C3ED94FE32
:101CB000601950CEBD0029EC600F7520007521FF22
:101CC000752900752A000200008100A827A92808AC
:101CD00009D804D90281DDB191EAF281D10D81A642
:101CE000C3ED94035051EDA2E092007AC5C3E582A2
:101CF0009400E583941C508C200010438F02438F86
:101D0000018529B7852AB7F0300027A827A9280818
:101D100009438F01538FFDD804D902A132C3E58353
:101D2000941C4003A3A117E28529B7852AB7F0A325
:101D3000A117538FFC81827AC1BD030CE493A3FAEF
:101D4000B152DCF8B14A81828184AA22AB23B16E00
:101D5000EBFAEA6222752608C3E52313F523E52290
:101D600013F52250066323A0632201D526EAB1DBD6
:101D7000B1DB75260AEAF4200102D284300102C2E6
:101D800084B1DBC3134002C201D526EB22B191EA34
:101D9000FB208402A191308402A196752608AE240E
:101DA000AF25C3EF13FFEE13FEB1DFB1DBC3EA13C0
:101DB0003084024480FA30E703632201C3E5231331
:101DC000F523E52213F52250066323A0632201D5F3
:101DD00026D9E52265236523F52222AE24AF250E00
:101DE0000FDEFEDFFCD20122424C48656C693437BD
:061DF0003164E8B10601B8
:00000001FF
